:020000020000FC
:1000000064CEBCC10000000020C000008EC0000013
:10001000000098C000000000000000000203040679
:10002000080C10182030406080000406080C1018DE
:100030002030406080A0C0000003070F1F000D0D9E
:100040000403060D0503030202004FB662FD0CC057
:10005000552041F00994C52DC095089483FDC7959E
:10006000C4BD64604FBE1895C0916400089483FDC0
:10007000C795C4BD6B7FC0916400CF3F09F41EC01B
:1000800070FF1AC082FD05C04FBE9198909893985A
:10009000189576FD0EC065FD0CC0C091B100C0FD85
:1000A0009498C1FD9798C2FD9598CAEFC095CA95DE
:1000B000F1F79198909893984FBE189524BCCC274F
:1000C000C064C8BF6460F8CFC6CF70FFC4CF65FD01
:1000D000C2CF919AC0CF70FFBECF65FDBCCF909AC2
:1000E000BACF70FFB8CF65FDB6CF939AB4CF949ACC
:1000F00070FFB1CF65FDAFCFC7E0CA95F1F7919A18
:10010000AACF979A70FFA7CF65FDA5CFC7E0CA9584
:10011000F1F7909AA0CF959A70FF9DCF65FD9BCF88
:10012000C7E0CA95F1F7939A96CF4FB6C9B7CF7E7D
:10013000C9BF6E7FCCB5CE0DDDB5DF1DDBBDCABD41
:100140004FBE18953FB68F7EABB7A074A2118061E9
:10015000A0E0ABBFA9B7AE7FA9BF7894A09168001B
:10016000AA2341F085FD2AC0A0916800AA95A0931A
:10017000680024C040E050E085FD14C0A0B396FDA7
:10018000A095A2FD4FEFA3E096FDA2E0A5BFAA2790
:10019000A064AABF8D7FA0B396FDA095A2FD5FEFDE
:1001A000451741F7A0E461FDA093680085FD03C0F9
:1001B000A0E4A093680040939600816085FD0EC086
:1001C000A0916900AA2331F0A0916900AA95A0939B
:1001D000690004C08061AA27A064AABF80FF0AC08A
:1001E000A09196004A2F61FF8E7F85FD01C000C05F
:1001F000409361004091B400443009F004C0A091E4
:100200006100A0936300A52DA03408F06860A09160
:100210006000A395A093600051F0F894A9B7A16085
:10022000A9BF84FF02C0A0E4ABBF3FBE1895A09158
:100230007400A395A093740042E050916800552388
:1002400029F085FF03C05A9550936800A09196004D
:10025000A13018F0209299000DC020929A002092AF
:10026000A300A0919900AF5FA093990018F0AFEFA1
:10027000A0939900B09061005091B400523049F4BD
:1002800066FF91F0A2E3BA1678F0A0918600A093E1
:100290006100533049F466FF39F0A2E3BA1620F04A
:1002A000A091C000A0936100509162005B1521F005
:1002B00010F05A9501C05395509362004A95D1F6BB
:1002C0005091A300539509F45A955093A300A0911F
:1002D000A400AA95A093A40009F046C0A1E0A093B1
:1002E000A40045E0A091A5005A17F0F1A091A60046
:1002F0005A1728F441E0A3E0A093A40007C0A091FE
:10030000A7005A1718F441E04093A400D0909C0035
:10031000C0906300DC14A8F0A091B400A430D9F020
:1003200066FD0FC0C0929C00539511F0A091A500EE
:10033000A093A300A1E0A093A400ACE3A09362006B
:1003400013C0A0919C00A40F20F45FEF50939C0079
:1003500002C0A0939C00A0919C00AF3F29F4AFEF96
:10036000A0939A00A093A300F894A9B7A160A9BF95
:1003700084FF02C0A0E4ABBF3FBE18953FB64CB5AA
:100380005DB58F7EABB7A074A2118061A0E0ABBF5A
:10039000A9B7AE7FA9BF789481FD23C0A2E096FDE6
:1003A000A3E0A5BF8260A0B396FDA095A2FF05C003
:1003B00040936500509366001CC1A3E096FDA2E047
:1003C000A5BFAA27A064AABF8D7F85FF01C004C175
:1003D00040E0A0B396FDA095A2FDFEC0409396001C
:1003E000EDC0A3E096FDA2E0A5BF8D7F61FF71C0C7
:1003F000A2E096FDA3E0A5BFAA27A064AABF8260E1
:100400004093910050939200A0908F004A19B090B1
:1004100090005B09BB24A22C4C38520518F42092A2
:10042000950049C0A091D400AA2359F1483C520537
:1004300028F4A0E1BA2EAAE0AA2E23C04836A1E0F3
:100440005A0728F4A8E0BA2EAFE0AA2E1AC0403D01
:10045000A2E05A0728F4A4E0BA2EAEE1AA2E11C0F9
:10046000403AA5E05A0728F4A2E0BA2EACE3AA2E3F
:1004700008C04839A8E05A0720F4A1E0BA2EA8E73E
:10048000AA2EC42EA0919300CA1AD52EA091940032
:10049000DA0ADD202AF4AFEFC094D094CA1ADA0A3F
:1004A00020929500A8E0A210A0E0CA14DA0618F481
:1004B000A1E0A09395004093930050939400409145
:1004C00091005091920040938F005093900042E031
:1004D00075C0A09165004A1BA09166005A0B94FD5F
:1004E00060C093FD5EC092FD5AC086FF03C0D52E4A
:1004F000C42E0CC05695479591FD51C05695479511
:1005000090FD4DC0D52EC42ED694C79461FD19C060
:10051000AC2DAC51AD2DA24008F005C0DD2089F412
:10052000AC2DA85C70F4A0916700A395AA2311F0EC
:10053000A0936700AA3008F44FC020929600816013
:100540004BC0A0916700AA2319F0AA95A093670059
:10055000A22C5091BA0097FD02C0A090C800AAEF4B
:10056000AA0EA22DA21DCA18DA0A4FB74170442361
:1005700019F040E050E015C0AFEFCA16D20418F0F1
:100580004FEF50E00EC0A091AC00CA9E412D000C70
:10059000441F50E008F012C04FEF50E00FC05695D6
:1005A000479594FF07C0552309F04FEFA42FA69558
:1005B0004A0F521D4F3F520508F04FEF40939600EF
:1005C000816061FF09C0AFE1A095A923AB299A2FF3
:1005D0008F7DBB2009F48062A0E4A093680085FFB2
:1005E00003C0AAE0A093680061FD03C085FD01C0BF
:1005F0008F7E85FD03C0A0E2A0936900F894A9B79F
:10060000A160A9BF84FF02C0A0E4ABBF3FBE1895A4
:1006100011E00AC013E008C01AE006C01EE104C0E1
:1006200014E602C018EC00C005E1BB27BA95F1F74B
:100630000A95D9F71A95C1F708952AE338E709C052
:1006400020E33CE806C02AE234EB03C025E238ECA4
:1006500000C012E0BB27979ABA95F1F7909ABA9525
:10066000F1F79098BA95F1F79798BA95F1F712309B
:1006700009F0919A123009F4939AB091AD00BA95AD
:10068000F1F7123009F09198123009F49398B7E815
:10069000BA95F1F71A95F1F6022FB22FBA95F1F744
:1006A0000A95D9F73A95A9F6979A0895221B39E049
:1006B000001F3A9509F40895221F211B18F4210FF9
:1006C0008894F6CF0894F4CF622C722CB0E0889412
:1006D000B395221F331FE0F7379527958894912E05
:1006E000802E020B130B10F4192D082D10F4889492
:1006F00001C00894661C771CBA9571F7172D062D5A
:100700000895322D11232AF43A9500951095031B74
:10071000130BF894029F712C002D129F912C802CAA
:100720007894780C172D921C292DB4E06B2E269509
:10073000179507956A94D9F7332321F00095109502
:10074000031B130B08950091B400043009F474C026
:10075000B0919600B95198F0B72FB67081F466FD4C
:100760002BC005E09090C600B92DBA9521F00AE0A3
:10077000BA9509F002E1B0917B00B01BE0F066FF92
:100780000AC0B0919E00B0939C00BFEFB093A3004D
:10079000B1E0B093A400B0916100B09363002092E7
:1007A0007E0020927F002092800020928100209283
:1007B00082006F7B41C060649090C600B92DBA95ED
:1007C00079F4B0916200B095BB1FBB1F1B2FB7958A
:1007D0000B2FB12FB170B3951B2FB02FBE7F25C04B
:1007E000B92DBA95BA9581F4B0916200B095BB1F4E
:1007F000BB1FBB1F1B2FB7950B2FB12FB370B3952A
:100800001B2FB02FBC7F14C0B0916200B095BB1FEE
:10081000BB1FBB1FBB1F1B2FB7950B2FB12FB77073
:10082000B395B3951B2FB02FB87FB0540B2F12097F
:1008300000937E0010937F00089510917B00169521
:1008400000917A000795B0917E00B01B0B2FB091FC
:100850007F00B10B1B2F28F40038BFEF1B0740F0BF
:1008600009C00F37120508F405C00FE710E002C0F9
:1008700000E81FEF00938300109384000895009117
:100880008300B09180000B0F10918400B091810023
:100890001B1F20E03091840033230AF42A95B09185
:1008A00082002B1F1AF4203F40F00AC02F3008F4BA
:1008B00007C00FEF1FEF2FE003C000E010E020EFB4
:1008C00030916300B0919B003B1718F4323030F048
:1008D00009C0B0918400BB235AF004C0B0918400D9
:1008E000BB2332F400938000109381002093820098
:1008F00008952091D70000918300000F109184008B
:10090000111FFFDE11232AF40038BFEF1B0740F050
:1009100009C00F37120508F405C00FE710E002C048
:1009200000E81FEF002352F0B0916200B01B0B2FC4
:1009300018F0013008F00AC001E008C000950F5F10
:10094000B09162000B0F08F001C00FEF009385001B
:1009500008952091D8000091810010918200D1DE8D
:1009600011232AF40130BFEF1B0740F009C00F3FED
:10097000120508F405C00FEF10E002C001E01FEF00
:10098000112352F0B0918500B01B0B2F18F00130ED
:1009900008F00AC001E008C000950F5FB091850023
:1009A0000B0F08F001C00FEF0093630008950FEFE5
:1009B000677F71FD29C072FD09C06860B0917B003E
:1009C000BA3020F0B52DB03408F4677FB091D30071
:1009D000BB23D1F0B0917B00BB23B1F00FEF10919E
:1009E0007B0064DEF894B091730072FDB5E00B9F5C
:1009F000112D002D7894112309F00FEFB0919E0076
:100A00000B1710F400919E0000939D000895009133
:100A10007A0010917B0000541140B0919D0010F4B9
:100A2000BA9501C0B39511F0B0939D000895E7D336
:100A3000B7E074FDB7E0B06CB7B9B6B1B068B064F8
:100A4000B6B9E6DDB7E074FDB7E0B06CB7B9B6B1E2
:100A5000B068B064B6B9B6B1B6FDFDCF04B115B19A
:100A6000B6B1BF77B6B922D420E02093A8002223E4
:100A700009F441C030E03093A900732E7694622EC1
:100A80006694620E731E262D372D0217130778F019
:100A90008090A800B0E0B80DB093A8008090A900A5
:100AA000B0E0B81DB093A900260D371DEECF8090A1
:100AB000A8009090A9001091A90016950091A80097
:100AC00007951695079523E0169507952A95E1F762
:100AD0002091B5002A9529F42092A8002092A9001F
:100AE0000AC02A9521F0800E911E2A95E1F7809286
:100AF000A8009092A90008952091B500B6B1B6FD66
:100B0000FBCF04B115B1B6B1BF77B6B9B091AA00A9
:100B1000B395B093AA00B83060F12092AA00B091CA
:100B2000D200BB2321F1112329F0B091AB00BF3FCC
:100B300061F009C0B091AB000B1739F020F4BB2372
:100B400021F0BA9502C0B395E1F300919B00B093F8
:100B5000AB00B03050F400ECB03038F400E8B03006
:100B600020F400E4B03008F400E000939B007F7EA6
:100B700008952130B1F00F3FB3E01B0790F4B0E0CF
:100B8000BB2379F0B091A8000B17B091A9001B0707
:100B900040F4B0919B00BB2359F0BA95B0939B00F1
:100BA00007C0B0919B00BF3F19F0B395B0939B0075
:100BB00000919B00B0916300B01B10F400916300A2
:100BC000B0919C000B1750F000919C00B0919C00DC
:100BD000BF3F21F0B0919C00B0939B00502E00933A
:100BE0006400B091AA00B73009F47061089502E37F
:100BF000F894B091D9000B9F012D000C001F789440
:100C0000B0919B000B1710F000919B0000936100C6
:100C100000936300502E0093640000939E0008959B
:100C200020927A00B0EFB0937B000895F8940CB551
:100C30001DB5209174007894309175006090760015
:100C40000093750010937600031B160971FD03C015
:100C500077FD7DC027C0709077002093770027092B
:100C6000222311F00FEF1FEF809078009090790011
:100C700030937800609279000091750010917600B1
:100C80000819190920917A0030917B003695279533
:100C9000020F131F10F40FEF1FEF00937A00109351
:100CA0007B0029C020917A0030917B003901B4E0AB
:100CB0008B2EB2E09B2E343010F08A949A94383008
:100CC00010F08A949A94769467948A94E1F726199E
:100CD0003709992021F0169507959A94E1F7200F8E
:100CE000311F20937A0030937B0028F43FEF30933C
:100CF0007A0030937B00323008F4706871FF02C0D4
:100D0000B3E00DC0B091C40000917100023838F01A
:100D1000B395003A08F0B395B63008F0B5E09B2ED5
:100D2000B4E08B2E10917B0000917A0024E01695A0
:100D300007952A95E1F70819120928F0B02FB2504B
:100D4000B12FB20910F402E010E0980126C0209102
:100D50007A0030917B0039017694679466946694AA
:100D600066942619320906950695200F321D2093A8
:100D70007A0030937B00323008F07F7704E03695BC
:100D800027953695279526952695201B10F022301D
:100D900008F422E089019090C40060FDFECFE0904D
:100DA0008B00F0908C006160B9B7B061B9BF3801B9
:100DB00077FD41C07694679400938B0010938C006C
:100DC000B92DB330E1F0B0FD04C0060D171D93013D
:100DD00006C0000F111F0250120922E030E0B92DA9
:100DE000B33068F020938D0030938E00009387001D
:100DF000109388006092890070928A003AC0009334
:100E00008D0010938E0020938700309388006092AD
:100E1000890070928A0071FF0DC0BFE0B0938D0011
:100E200020928E00B093890020928A00B0938B00AC
:100E300020928C001EC0669400938B00B92DB330B5
:100E400091F0B0FD03C0060D262D03C0000F025027
:100E500022E0B92DB33038F020938D000093870045
:100E60006092890006C000938D00209387006092F5
:100E7000890000917C0002FD0350013031F495FDA2
:100E80000CC0B2E0B06CB7B90BC0023021F4B3E0D3
:100E9000B06CB7B905C095FDF4CFB4E0B06CB7B98C
:100EA0000091A200000F10F4BBE60B270093A200F4
:100EB00060FDFECFB2E0B0936E006160B9B7B06183
:100EC000B9BFB72FB670D1F020917A0030917B0076
:100ED000369527953695279571FF02C0B0E43B0FF4
:100EE000F8940CB51DB5020F131F1BBD0ABD616040
:100EF000B0E1B8BFB9B7B061B9BF78940895606187
:100F000020927D0020E067FD20E206C06061209213
:100F10007D0020E267FD20E001E011E077FD11C0D7
:100F2000B72FB67009F06F7E14E100917B00069533
:100F300009F403950F3008F00FE071FF02C004E1DF
:100F400014E160FD0FC0B0917D00BB2359F071FF2B
:100F500006C0B0916E00BA95B0936E0011F4706245
:100F600047C0ABDFB0B7B77FB0BFB8B1B0B7B860FC
:100F7000B0BFB0917D00B395B0937D00B8B177FD5F
:100F800006C0B1E071FDB3E0BA95F1F7B8B1B07247
:100F9000B21709F022C071FF05C00395011708F0D0
:100FA0000A95CFCF64FD05C00395011708F0B4CFB3
:100FB000C8CF6F7EF8943CB56DB470907A00809085
:100FC0007B00370D681C6BBC3ABD6160B0E1B8BFF7
:100FD000B9B7B061B9BF78949FCFB0916D00B1300F
:100FE00008F49ACF64FD98CF0A9509F0AACF7F7DC7
:100FF00020918D0030918E00F894B0E1B8BF0CB50F
:101000001DB5020F131F1BBD0ABDE0908700F090B5
:1010100088006160B9B7B061B9BF7894B72FB67076
:1010200039F0B0916D0072FFB395B0936D0009C0B7
:1010300075FF07C067FD05C064FD03C0BF91BF9188
:10104000EBC4089500E063FF03C064FF01C001E04A
:10105000F89410917100B7E01B9F212D102D78940A
:10106000200F269517952695179526951795109379
:101070007100183718F4B8E7B0937100009171004F
:10108000B09172000B1720F060629198909893983D
:1010900060FDFECFE0908900F0908A006160B9B7F2
:1010A000B061B9BF0895B2E095FD0AC0F894B0935D
:1010B0007C00979A949862FF01C0939A7894F4C048
:1010C000F894B0937C00979A959862FF01C0919A2A
:1010D0007894EAC0B3E082FF24C095FD11C002E01D
:1010E000F894B0937C00E1E8F0E00093B1009398AD
:1010F000959A62FF02C0909A01C097987894D4C0E4
:1011000002E0F894B0937C00E1E8F0E00093B100D5
:101110009198949A62FF02C0909A01C0979878942F
:10112000C3C095FD0BC0F894B0937C00EBE6F0E0F3
:10113000939862FF01C0909A7894B6C0F894B093E7
:101140007C00EBE6F0E0919862FF01C0909A789401
:10115000ABC0B4E095FD0AC0F894B0937C00949ABB
:10116000959862FF01C0909A78949EC0F894B093CD
:101170007C00959A949862FF01C0909A789494C0EC
:10118000B5E082FF24C095FD11C001E0F894B09352
:101190007C00E7E7F0E00093B1009098979A62FF37
:1011A00002C0919A01C0949878947EC004E0F894AB
:1011B000B0937C00EBE8F0E00093B1009098979A30
:1011C00062FF02C0939A01C0959878946DC095FD16
:1011D0000BC0F894B0937C00E5E6F0E0909862FFD5
:1011E00001C0919A789460C0F894B0937C00E1E7D4
:1011F000F0E0909862FF01C0939A789455C0B6E0F1
:1012000095FD0AC0F894B0937C00959A979862FF78
:1012100001C0919A789448C0F894B0937C00949A55
:10122000979862FF01C0939A78943EC0B1E082FF24
:1012300024C095FD11C004E0F894B0937C00EBE865
:10124000F0E00093B1009198949A62FF02C0939AE3
:1012500001C09598789428C001E0F894B0937C0080
:10126000E7E7F0E00093B1009398959A62FF02C01F
:10127000919A01C09498789417C095FD0BC0F8948A
:10128000B0937C00E1E7F0E0919862FF01C0939A8F
:1012900078940AC0F894B0937C00E5E6F0E0939867
:1012A00062FF01C0919A78946F7D089524E630E042
:1012B000F9012092B100919890989398949A979AF6
:1012C000959A6B7F0895A2EBB0E007E00D9307E0DD
:1012D0000D9301E00D9304E00D930FEF0D930D932B
:1012E00009E00D9302E00D9301E00D9301E00D93F1
:1012F000AEEBB0E001E00D9300E00D9304EB0D9335
:101300000FEF0D930D930D9303E00D930FEF0D93DE
:1013100001E00D930FEF0D9305E20D9300ED0D939A
:1013200008E70D9308EC0D9304E00D930FEF0D9378
:1013300001E00D9300E00D930AE70D930AE00D9391
:1013400000E00D9301E00D9300E00D930FEF0D937E
:1013500000E00D9308952091B9008B7F233009F4AC
:101360008460B091BA009F7DB1FD90629F7BB09187
:10137000BB00B1FD9064223011F0886001C0877F0E
:1013800008950A95E00FF21DB4910895ECE1F0E0A4
:101390000091B200F6DFB093D700ECE1F0E00091ED
:1013A000B300EFDFB093D800EAE2F0E00091B800BC
:1013B000E8DFB093D9000091D100002309F4039530
:1013C000013108F001E1B02FB00FB00FB093A500CC
:1013D0001B2FB10FB10FB00FB093A600B10FB00F1C
:1013E000B00FB093A7000091B800023008F402E0FB
:1013F00000937300B091CE000FEFB23009F400EA11
:10140000B33009F402E800937200E8E3F0E00091E1
:10141000D500B7DFB093A000089508952091C800CB
:101420003091C900B091BA00B33009F43E5097FF33
:1014300002C020E03FEFB32FB21B6B2EB25810F466
:10144000B2E86B2E00E00395609EB12DBD57D8F336
:101450000093AC0008959068E1DFE0D820E030E030
:10146000B0E16B2ED7D8B09196002B0F321D6A9445
:10147000C9F7B4E036952795BA95E1F7822E9F77A4
:10148000CDDF0895F894E3E0F0E0B9E0B7BFB491A0
:10149000B078C1F3F894A895B1B5B861B1BDB0E02A
:1014A000B1BDB4E0BEBFBFE5BDBF00DFB0E0B8BBBB
:1014B000B0E1B7BBB0E0B5BBB0E0B4BBB0EBB2BB22
:1014C000BBEBB1BB2224A0E0B0E02D92AA31E9F73A
:1014D000A0E6B0E00FEF2D920A95E9F7B1E0B093E6
:1014E000A200F1DEDAD2B7E0B06CB7B9B6B1B46041
:1014F000B068B6B90091CA000093AD00B1E0B093F6
:101500006A00F8948FD899D889D89AD887D89BD868
:1015100085D852D387D886D883D8F8940AEF1AEFA3
:10152000A0B396FDA095A2FF1FC01A95C9F70A9512
:10153000B1F7E0E0FCE1B591B43E39F4B591B03ECD
:1015400021F4B591BF3F09F40CC0E0E0F395F395A9
:10155000B591B83F49F4B591B43931F4B591BA3A7F
:1015600019F4EE27F6950994F6DE10DF56DF56DF04
:101570000091CA000093AD0099DEB2E0B3BFB2E0C3
:10158000BEBDB2E0B5BDB1E5B8BFB9BFB0B7B77FBA
:10159000B0BFB8B1B0B7B860B0BF3AD8789447DA46
:1015A00020927000B3E096FDB2E0B5BFB0E4BBBFDF
:1015B000BB27B064BABF8D7F35D8626033E02CE0C2
:1015C000B0919500BB2321F42CE03A9509F4A5CF06
:1015D00025D880FFA2CF8E7FB0919600B23078F3ED
:1015E000B92FBF710091980000939700B0939800B5
:1015F000B01729F72A9521F76D7FB3E096FDB2E089
:10160000B5BFBB27B064BABF8D7FB091D400BB23F8
:1016100021F48062B92FB0709B2F8F7B20926700DE
:10162000FFD785FF05C0B0916700BA3008F080642D
:10163000F1D702E085FF01C000E0B0919600B0173D
:10164000B8F3F894FAD7F9D7F8D77894EBD7209273
:101650008600E0D7B091BE00B13008F46EC0B09102
:101660006A00B13008F469C085FD18C0B0919600D9
:10167000BF3F08F462C0F894E9D77894D1D7B0910D
:101680009600B130C0F7F894D8D7C6D7D6D778949B
:10169000C7D7B0919600BF3FB0F3C0C2B8E09B2E51
:1016A0009068F894BBDE7894BBD7F8949F77B6DE49
:1016B00080909600B0919600BF37789408F445C0AA
:1016C000A7D7F894C3D778949A9451F7C4DEB82D6D
:1016D000B550B093C900A6D7F8940CD272D27894C2
:1016E000BAE09B2E9068F89499DE789499D7F89494
:1016F0009F7794DE80909600B0919600BF377894E3
:1017000078F786D7F89499D787D797D778949A940B
:1017100049F7A1DEB82DBB5FB093C80083D7F8941A
:10172000E9D15ED278947CD7F89478DE7894B09141
:101730009600BF3F08F498CF71C200919600B09117
:1017400086000B1710F0009386006AD701E0B09175
:10175000BA00B35009F405E0B0919600B01708F054
:1017600078CFF89473D772D771D778945BD72092DB
:101770006A0020926B0020926C00B0916B00B395D0
:10178000B0936B00BF3F71F5B0916C00B395B0930F
:101790006C00B091CC0009E1BA9559F002E3BA951A
:1017A00041F00DE7BA9529F00AEFBA9511F02092B1
:1017B0006C00B0916C00B017A8F078DD29D7B0911B
:1017C0006C00BA95B0936C0020926B00B091CB0086
:1017D000B093AD00F8943AD77894B091CA00B09322
:1017E000AD001ED719D7B0916800BB2319F485FF4F
:1017F00001C093CE01E085FD01C006E0B0919600E6
:10180000B01708F4BACF0CD7B0916800BB2309F425
:1018100084CEF8944BDD20926100209262002092E9
:101820006300522C209264002092A1007894B09121
:10183000B700BB0FB0939F0020927E0020927F00E4
:101840002092800020928100209282002092AA00A3
:1018500060E070E020927100B8E0B093AA0070617F
:10186000D7D6B7E074FDB7E0B06CB7B9B6B1B06821
:10187000B064B6B9B6B1B6FDFDCF04B115B1B6B11D
:10188000BF77B6B9112309F00FEF0093AB0034D93D
:10189000B8E0B093AA0070615EDDF894BFEFB0933A
:1018A0009B00A5D9B0916100B0939B00B0939C00C0
:1018B000B0939D007894B1E0B0936100B093630061
:1018C0005B2EB0936400B093A400B0919A00B093E3
:1018D000A300B091BA00B33019F49F7D87FD9062E8
:1018E0007160726020926D008ADCA0DC99D99ED96B
:1018F00097D99CD995D90ADB26D7A4DBD4DB96D916
:10190000FEDA66FD9AD777FF52D877FD80D89ADB4A
:10191000E1DB8CD9FBDA66FDB2D794DB1ADC86D921
:10192000EEDA66FDE6D78EDB2BDC80D9EFDA66FDDA
:1019300010D888DB64DC7AD9E2DAB7E074FDB7E06E
:10194000B06CB7B9B6B1B068B064B6B97BDB6EDC69
:101950006DD9D2D871FF1EC0B0919E00B0939B008C
:10196000B0939C00B0919A00B093A300B1E0B09303
:10197000A40018E12CE0B0916D00B11728F07D7F34
:10198000746020936F0006C0B0919600B13008F0EB
:10199000B2CF4CC072FF11C067FD0FC0B0916F0095
:1019A000BA9519F47B7F7860A6CFB0936F00B091A1
:1019B0009600B13008F09FCF39C020927000B091EE
:1019C0009900B13058F0B0919E00B0939C00B09156
:1019D0009A00B093A300B1E0B093A400B091990035
:1019E0000AEF1091D600112309F003E0B01708F0B8
:1019F0001DC085FF04C0B0916800BB23B9F000EFA3
:101A000067FF05C0B0919E00B0939B0000E2B091CB
:101A10007B00B01708F46FCFB0917000B395B0930E
:101A20007000B0919600BB2309F002C020927000B4
:101A3000F8943CDC8090B900B2E0B093B9008BDC44
:101A40008092B9002092610020926200209263008F
:101A5000522C2092640020929F0060E070E0789405
:101A6000DFD524DC0091D600002319F0919A909ADA
:101A7000939AB7E0B06CB7B9B6B1B460B068B6B914
:101A800085FF05C0B0916800BB2309F446CDB09135
:101A9000BF00B13008F0CCCD6CCEEDE0F0E023D04B
:101AA000053A09F01BC0EEE0F0E01DD00A3509F060
:101AB00015C03AE0A2EBB0E0E3E0F0E014D00D9303
:101AC00031963A95D9F739E1AEEBB0E0EFE0F0E0CE
:101AD0000AD00D9331963A95D9F702C0F4DB0AD0BB
:101AE000E8E2F0E00895E199FECFEEBBFFBBE09A9B
:101AF0000DB308951ED03AE0A2EBB0E0E3E0F0E0D1
:101B00000D910FD031963A95D9F739E1AEEBB0E0AF
:101B1000EFE0F0E00D9105D031963A95D9F712D06B
:101B20000895E199FECF0DBBEEBBFFBBE29AE19AAF
:101B30000895EDE0F0E00FEFF4DFEEE0F0E00FEFFE
:101B4000F0DF0895EDE0F0E005EAEBDFEEE0F0E035
:101B50000AE5E7DF08953091AE000091AF00313023
:101B600011F40093B200323011F40093B30033301B
:101B700011F40093B400343011F40093C6003530F2
:101B800011F40093B500363011F40093B8003730EB
:101B900011F40093C400383011F40093B9003930C7
:101BA00011F40093CE003A3011F40093BA003B30A8
:101BB00011F40093BB00089525E034D52A95E9F788
:101BC00008953BD53DD53FD541D526D536D538D519
:101BD0003AD53CD521D531D533D535D537D508952E
:101BE00035D531D52DD529D517D530D52CD528D5F6
:101BF00024D512D52BD527D523D51FD50895809070
:101C0000AE009090AF0019D518D517D505D58A9498
:101C1000D1F71CD501D59A94E1F70895F894D1DF56
:101C20007894CADFC9DFB1E0B093AE00B1E0B09301
:101C3000AF002092B000F894E2DF7894B5E06B2E0C
:101C400070909600EFD4B09196007B16C9F7B13032
:101C500018F0BF3F40F107C07EDFF8944BDFB1DFE3
:101C6000B8E0B1BDA9DF6A9459F7B091B000B3955F
:101C7000B093B000B33008F4DECF9EDFB091AF0078
:101C8000B395B093AF00F894B091AE00BA95EEE37F
:101C9000F0E0EB0FF21D049178940395B091AF0042
:101CA000B01708F4C6CF88DF87DFB091AE00B395D8
:101CB000B093AE00B091AE00BC3008F4B7CF03DBF8
:0C1CC000F89418DFB8E0B1BD77DFDCCB92
:00000001FF
